:1000000012C01FC01EC087C01CC041C01BC0BAC2E6
:10001000E2C217C016C015C014C013C012C011C070
:1000200010C00FC00EC011241FBECFEDCDBF20E009
:10003000A0E6B0E001C01D92A139B207E1F76CD192
:100040007EC3DECF1F920F920FB60F9211248F93B3
:100050009F93AF93BF9380917D0090917E00A0917C
:100060007F00B09180000196A11DB11D80937D009D
:1000700090937E00A0937F00B0938000BF91AF91DA
:100080009F918F910F900FBE0F901F9018951F9208
:100090000F920FB60F9211248F939F93AF93BF933C
:1000A00080918D0090918E00A0918F00B091900072
:1000B0000196A11DB11D80938D0090938E00A09399
:1000C0008F00B093900080918C00882331F0809154
:1000D0008C00815080938C0001C0959A809185009E
:1000E00090918600892B49F080918500909186003F
:1000F0000197909386008093850080918C008C34CA
:1001000009F4C398BF91AF919F918F910F900FBE4B
:100110000F901F9018951F920F920FB60F921124F7
:100120000F931F932F933F934F935F936F937F93FF
:100130008F939F93AF93BF9322B712BE80917D00A0
:1001400090917E00A0917F00B091800010927D0080
:1001500010927E0010927F0010928000BA2FA92F7B
:10016000982F8827822B8093870090938800A093F4
:100170008900B0938A0080918D0090918E00A091AB
:100180008F00B091900044B555B5DC0199278827C0
:1001900060E070E0842B952BA62BB72B409160007C
:1001A0005091610060916200709163008C019D012B
:1001B000041B150B260B370B009381001093820054
:1001C00020938300309384008093600090936100BB
:1001D000A0936200B093630081E080938B0088EE6F
:1001E00093E09093860080938500C39A939883EC64
:1001F00099E00197F1F700C00000959883EC99E031
:100200000197F1F700C00000939A89E980938C0070
:10021000BF91AF919F918F917F916F915F914F911E
:100220003F912F911F910F910F900FBE0F901F9034
:1002300018959C01C29890E137FF02C0C19A01C095
:10024000C19883E08A95F1F70000C09A83E08A950F
:10025000F1F70000C09883E08A95F1F70000220FC3
:10026000331F915049F7C29A08957F928F929F92BF
:10027000AF92BF92CF92DF92EF92FF920F931F93B4
:10028000CF93DF93742E6B017C01C1148AECD806E6
:100290008AE9E8068BE3F80640F0CC24CA9429ECFE
:1002A000D22E2AE9E22E2BE3F22EC1E0D0E09AE032
:1002B000892E912CA12CB12C1C2F00277C120AC056
:1002C000C701B601A5019401ABD1CB018068802B99
:1002D000912B08C0C701B601A5019401A1D1C801A5
:1002E000862B972BA6DFC701B601A501940198D1F3
:1002F00069017A012196C930D105F1F6DF91CF91DC
:100300001F910F91FF90EF90DF90CF90BF90AF9033
:100310009F908F907F900895CF93DF93CDB7DD2787
:10032000C550CDBF0FE312E42FE001501040204034
:10033000E1F700C0000081B3886281BB82B38065B1
:1003400082BB87B3876087BBBB9AC29A10BE83B754
:10035000876083BF89B7826089BF1FBC8EB581600B
:100360008EBD8EB580648EBD12BC89B7886889BF8A
:1003700080E090E05EDF80E09CE05BDF80E090E08A
:1003800058DF80E09FE055DF81E09CE052DF8FEF97
:1003900099E04FDF82E09AE04CDF87E09BE049DFA5
:1003A00010927D0010927E0010927F0010928000CB
:1003B00010928D0010928E0010928F00109290007B
:1003C00010928700109288001092890010928A0083
:1003D000109281001092820010928300109284008B
:1003E00010928C0010928B008AE090E0909386002F
:1003F000809385007894959A939883EC99E001977F
:10040000F1F700C00000939A80918B00813031F0A9
:100410008091850090918600892BB1F740908700EC
:10042000509088006090890070908A00E090810070
:10043000F09082000091830010918400E982FA829A
:100440000B831C8310928B00EF28E02AE12A41F4F1
:1004500081E090E0A0E0B0E089839A83AB83BC8325
:100460008091850090918600892B99F410928600E6
:10047000109285009FE9A6E8B1E09150A040B040FD
:10048000E1F700C00000412C512C320108E00D833F
:1004900030C01AE0411651046104710440F124E6B1
:1004A000421651046104710440F188EE481683E05D
:1004B00058066104710438F190E1491697E2590633
:1004C0006104710430F1A0EA4A16A6E85A06A1E0D8
:1004D0006A06710418F1B0E44B16B2E45B06BFE0A3
:1004E0006B06710400F102E00D832AE01FC018E0E2
:1004F0001D8320E836E948E91BC027E02D8320E46E
:1005000032E44FE015C086E08D8320EA36E841E012
:100510000FC095E09D8320E137E209C0A4E0AD83E0
:1005200028EE33E004C0B3E0BD8324E630E040E0D1
:1005300080E8A82E96E9B92E58E9C52ED12CE12CD9
:10054000F12C00E010E050E060E070E080E090E02E
:1005500089D0120123015101620184D0E980FA801F
:100560000B811C811701280157016201E12CF12C3C
:1005700000E010E0A7D0E42F4D81B9018E2F952F18
:1005800074DE42CF1F920F920FB60F9211242F9359
:100590008F939F93EF93FF938BB19CB18871E09100
:1005A0006600EF5FE37020916500E21739F0E09399
:1005B0006600F0E0E759FF4F908301C082E080932E
:1005C0006400FF91EF919F918F912F910F900FBE3B
:1005D0000F901F9018951F920F920FB60F92112433
:1005E0008F939F93EF93FF939091680080916700A2
:1005F000981761F0E0916700EF5FEF70E09367009C
:10060000F0E0E359FF4F80818CB901C05598FF910C
:10061000EF919F918F910F900FBE0F901F901895A3
:10062000A1E21A2EAA1BBB1BFD010DC0AA1FBB1FF6
:10063000EE1FFF1FA217B307E407F50720F0A21B68
:10064000B30BE40BF50B661F771F881F991F1A94D5
:1006500069F760957095809590959B01AC01BD01FF
:10066000CF010895DF93CF939F92A0E49A2E0024A8
:10067000D001E001F00116950795F794E794D7941F
:10068000C794B794A79448F41068A20FB31FC41F6F
:10069000D51FE61FF71F081E191E220F331F441F08
:1006A000551F661F771F881F991F9A9421F79D0178
:1006B000AE01BF01C00111249F90CF91DF91089539
:1006C000689401C0E8948F929F92CF93DF9305D0F6
:1006D000DF91CF919F908F90089588249924F40101
:1006E000E401B0E41B2ED401220F331F441F551F19
:1006F000661F771F881F991F881C991CEE1FFF1FFC
:10070000CC1FDD1FAA1FBB1F8A149B04EC05FD052F
:10071000CE05DF05A007B10748F08A189B08EC0951
:10072000FD09CE09DF09A00BB10B21601A94E1F697
:100730002EF49401AF01BE01CD01000C0895F89490
:02074000FFCFE9
:00000001FF
